S123C000546869732070726F6772616D20697320636F707972696768742031393934202040
S123C02062793A2020202020202020202020202020204772616E742042656174746965200D
S123C040202045646D6F6E746F6E2C2020414220202020202043616E6164612020202020D1
S123C0602D2D2D2D2D2D2D2D2D2D2D2D2D2D2D2D416C6C2072696768747320202020202062
S123C0807265736572766564212020546869732070726F6772616D206D6179206E6F742033
S123C0A0626520636F70696564206F72202020207573656420696E2077686F6C65206F72B8
S123C0C0696E207061727420776974686F75742074686520657870726573736564202020C6
S123C0E07772697474656E20636F6E73656E74206F662074686520617574686F722E20209E
S123C1002A20202043414C4C45522D494420202A00313939372C204D2E2042656E6F697498
S123C12020002A20496E697469616C697A696E67202A002A202020204E6F6D732120202094
S123C14020202A002A20417474656E74652020202020202A002A206427617070656C2E2E25
S123C1602E2020202A0043686F6978204E6F6D3A2020202300212020426164202045505272
S123C1804F4D20202100212043616C6C20466163746F727920210012151515151512008695
S123C1A040B710398E00FFBDCD518638B74000BDCD518601B74000BDCD51860FB74000BDA1
S123C1C0CD518606B740008640BDCD51B74000C608CEC197A60008BDCD375A26F78601BD04
S123C1E0CD51B74000BDCD571A8377C42716CEC175BDCD4086C0BDCD51B74000CEC186BD78
S123C200CD4020FECEC100BDCD4086C0BDCD51B74000CEC111BDCD40CE00C8BDCCB3092613
S123C220FA8601BDCD51B74000CEC122BDCD4086C0BDCD51B74000CEC133BDCD40CEB610F4
S123C240C60AA6008130240A8630BDCCC0BDCCD5200C813923088630BDCCC0BDCCD5085A58
S123C26026E0C610A6008120240A8620BDCCC0BDCCD5200C817F23088620BDCCC0BDCCD578
S123C280085A26E0A60027074FBDCCC0BDCCD5088CB7DB25AB8606B7102B4FB7102C860428
S123C2A0B7102D4F97049705970C970ECE000FDF08860197028600970D860197064FB71070
S123C2C0268640B710240EB6102E842026037EC669B6102FD60DC11623037EC39958CEC270
S123C2E0E63AEE006E00C314C331C373C3BCC3F3C422C447C470C484C499C4C8C4F0C56950
S123C300C590C5C4C5E0C399C399C399C399C609C61EC64081042609970A8601970D7EC6A9
S123C32069818027037EC669970A8607970D7EC6698109260D97079B0A970A8602970D7EEE
S123C340C358811227078600970D7EC66997079B0A970A8603B7000D9604810A25127A001F
S123C36004CE000FC6BDA615A700085A26F8DF087EC669813025228139221EDE08A7000858
S123C380DF089B0A970A7A00079607810127037EC6698604970D7EC6698600970DCE000F13
S123C3A096042706C6153A4A26FCDF087D000C2604C601D702960497057EC669813025300E
S123C3C08139222CDE08A70008DF089B0A970A7A00079607810A27037EC6698605970DDE02
S123C3E0088603A70008860AA70008DF087EC6697EC399814F2707815027037EC399DE0893
S123C400C604E70008C601E70008A70008DF089B0A970A7A000727037EC3998606970D7E9A
S123C420C6698130251E8139221ADE08A70008DF089B0A970A7A000727037EC669860697A2
S123C4400D7EC6697EC3999B0A27037EC3998600970D7D000C2604C601D70296044C97049D
S123C4609705CE000FC6153A4A26FCDF087EC669810D24037EC399970B9B0A970A8608978E
S123C4800D7EC669810127037EC3999B0A970A7A000B8609970D7EC669810827037EC39920
S123C4A097077A000B9B0A970A860A970D9604810A25127A0004CE000FC6BDA615A7000837
S123C4C05A26F8DF087EC669813025218139221DDE08A70008DF089B0A970A7A000B7A009B
S123C4E00727037EC669860B970D7EC6697EC3998102271381042724810627358107273F40
S123C500810827507EC399DE08A70008DF089B0A970A7A000B860C970D7EC669DE08A70086
S123C52008DF089B0A970A7A000B860E970D7EC6699B0A970A7A000B8614970D7EC669DEC4
S123C54008A70008DF089B0A970A7A000B8610970D7EC669DE08A70008DF089B0A970A7A4B
S123C560000B8612970D7EC6698107270B81082707810A27037EC399DE08A70008DF0897B0
S123C580077A000B9B0A970A860DB7000D7EC6698130252D81392229DE08A70008DF089BA2
S123C5A00A970A7A000B7A000727037EC6697D000B26078616970D7EC669860B970D7EC6D4
S123C5C0697EC399810127037EC399DE08A70008DF089B0A970A7A000B860F970D7EC66961
S123C5E0814F2707815027037EC399DE08A70008DF089B0A970A7A000B26078616970D7E32
S123C600C669860B970D7EC669810127037EC3999B0A970A7A000B8615970D7EC669814CFB
S123C6202707815227037EC3999B0A970A7A000B26078616970D7EC669860B970D7EC6692A
S123C6409B0A27037EC3998600970D7D000C2604C601D70296044C97049705CE000FC615DB
S123C6603A4A26FCDF087EC6697D000C27037EC6EB7D000126037EC6EB7D0002266DB610EC
S123C68008840426099605810123604A2010B610088402261796054C91042302204D970582
S123C6A0860197027F00007F0001203F7D0003273AB61008841026070F7F00037EC19FB663
S123C6C01008842026088601970C97022013B61008840826167D000427119605BDCA20865F
S123C6E00197027F00017F000320007D000C26447D0002273F7D000426298601BDCD51B7B9
S123C7004000860CBDCD51B74000CEC144BDCD4086C0BDCD51B74000CEC155BDCD407F008F
S123C7200220117F0002860CBDCD51B74000BDCB45BDCA5E960C810126697D000226647DF2
S123C7400001275FB610088402260996064C81112312204FB610088404261796064A8101B2
S123C7602402203F9706860197027F00017F000020317D00032717B610088420261086FF38
S123C780970C860197027F00017F00032015B610088418260E8602970C860197027F000132
S123C7A07F0003960C8101263F7D0002273A8601BDCD51B74000CEC166BDCD409606BDCD4C
S123C7C016BDCCEDBDCD3717BDCD3786C0BDCD51B74000CEB61AC61B96064A27033A20FA35
S123C7E0BDCD407F00022000960C81FF27037EC88D7D000227037EC88D7D000126037EC842
S123C8008DB6100884022606B640014C200BB6100884042644B640014AC610BDCD51F740B0
S123C82000F64000C440260E813024028639813923108630200C81202402867F817F230230
S123C8408620BDCD51B74001C610BDCD51F740007F0001863297002034B6100884082605CB
S123C860BDC9E920EB7D00032723B6100884102607BDCC0C86012008B610088420260E4FA8
S123C880970C4C97027F00017F00032000960C81FF2658960227547F00028601BDCD51B79D
S123C8A040008623BDCD379606BDCD16BDCCEDBDCD3717BDCD378620BDCD378620BDCD37B1
S123C8C0CEB610C61B96064A27033A20FABDCAE186C0BDCD51B74000BDCD408685BDCD514B
S123C8E0B74000860EBDCD51B74000960C810226709602276C7F00028601BDCD51B7400017
S123C900D60E4F8F960EBDCCEDBDCD3717BDCD37863ABDCD37C604378620BDCD37A6000807
S123C920BDCCEDBDCD3717BDCD37335A26E986C0BDCD51B740003C3332BDCCEDBDCD371741
S123C940BDCD37863ABDCD37C604378620BDCD37A60008BDCCEDBDCD3717BDCD37335A26B9
S123C960E9960C8102264A7D000226457D00012740B6100884022606960E8B08200BB610BE
S123C9800884042612960E8008970E860197027F00017F0000201A7D00032715B610088493
S123C9A020260E8600970C860197027F00017F0003B61008843E813E260C96038105220B07
S123C9C08B019703200A7F000320058601B700013E7EC2C78640B7102596008B01816426F9
S123C9E0054FC601D70197003B8614BDCD51B74000BDCD51B64000847F810726098614BD20
S123CA00CD51B7400039810F260986C0BDCD51B7400039815026088685BDCD51B74000399F
S123CA20B1000426107A00047A0005FC0008830015FD000839C615CE000F4A27033A20FAB0
S123CA40F60004F0000586153DA615A700085A26F87A0004FC0008830015FD000839A6002B
S123CA60810227248104270139C6C0BDCD51F740000808A600CECB23814F2708CECB3481A7
S123CA8050270139BDCD4039083C1838E60008C00A3ABDCC768C0000270C86C0BDCD51B7C2
S123CAA04000BDCD4039183C3886C4E600C107270E8001C10827088001C10A27028001BD4A
S123CAC0CD51B74000E60008C10A2715C10722022026A60008BDCD37862DBDCD37C1082347
S123CAE017A60008BDCD37A60008BDCD37A60008BDCD37862DBDCD37A60008BDCD37A60045
S123CB0008BDCD37A60008BDCD37A60008BDCD37A60008BDCD37A60008BDCD37A60008BD21
S123CB20CD37392A204F7574206F662052616E6765202A00204E756D65726F20507269768F
S123CB4065212020008601BDCD51B740008623BDCD37B600058B30813A26028600BDCD37A8
S123CB608620BDCD37BDCD37CE000FB60005C6154A27033A20FA0808A60008BDCD37A60029
S123CB80090909BDCD37862FBDCD37A60008BDCD37A600080808BDCD378620BDCD37E60004
S123CBA058585858A60180301B8112242CA6000881302703BDCD37A60008BDCD37863ABD86
S123CBC0CD37A60008BDCD37A60008BDCD378661BDCD37866DBDCD3739811227038B8819F1
S123CBE0BDCCED81302703BDCD3717BDCD370808863ABDCD37A60008BDCD37A60008BDCD0F
S123CC00378670BDCD37866DBDCD37390F8685BDCD51B74000CEB610C61B96064A27033A8A
S123CC2020FAC603BDCD51B64001A1002706BDCCC0BDCCD5085A26EC8689BDCD51B7400071
S123CC40C607BDCD51B64001A1002706BDCCC0BDCCD5085A26EC86C0BDCD51B74000C6105A
S123CC60BDCD51B64001A1002706BDCCC0BDCCD5085A26EC0E39183C3736F6B61018CEB695
S123CC80105D2727373C183CC60AA60018A100260F0818085A26F338C60A3A183833200E1C
S123CCA01838C61B183A38335A26D9CE00003233183839183C18CE06DA180926FC18383987
S123CCC0368616B7103BA7004CB7103BBDCCB34FB7103B3239368602B7103B3236A700863A
S123CCE003B7103BBDCCB34FB7103B32393C36CECD0616545454543AE60017CECD0633C4EB
S123CD000F3AE600383930313233343536373839414243444546373C16CECD223AA600386F
S123CD2033390001020304050607080910111213141516171819207D40002BFBB740013955
S123CD40A600084D2601397D40002BFBB7400120EF7D40002BFB39CEC00018CEC19E18FF84
S123CD60000818CECDC1CC0000FD00058601B70007A600B4000727028601F60006C47F18B8
S123CD803C183A18E6001838F70004B80004F60005595959F70004B8000444790006790003
S123CDA00574000725098601B10007270920C28680B7000720BBBC000827030820B3DC0527
S123CDC0390000010100000101010100000101000000000101000001010101000001010006
S123CDE0000101000001010000000001010000010101010000010100000000010100000120
S123CE000100000101000001010101000001010000000001010000010101010000010100FD
S123CE200001010000010100000000010100000101010100000101000000000101000001DF
S104CE4001EC
S123FFD6C19FC19FC19FC19FC19FC19FC19FC19FC19FC19FC19FC19FC19FC9D4C19FC19FCA
S10DFFF6C19FC19FC19FC19FC19F1D
S9030000FC
